:030000000219FDE5
:03000B000200A848
:03002B000201547B
:03005B000202D4CA
:030073000202C1C5
:1000800002030406080C10182030406080040608A3
:100090000C10182030406080A0C00003070F1F051F
:1000A000050D050205030302C2AFC0D0C0E0206207
:1000B00014E5256009E473E525F4F58AD262D0E001
:1000C000D0D0D2AF3285268AC262E526F46029D02C
:1000D000E0D0D0D293D295D297D2AF32D293D295EC
:1000E000D297206F0C2065097426D5E0FDE57B4290
:1000F00090D0E0D0D0D2AF32758A00C28DD26201EA
:10010000F101B7306805206502C29301B730680578
:10011000206502C29501B7306805206502C29701CB
:10012000B7C29230680A2065077430D5E0FDC293EB
:1001300001B7C29430680A2065077430D5E0FDC26B
:100140009501B7C29630680A2065077430D5E0FD86
:10015000C29701B7C2AFC2AD53E6EFC0D0C0E0D284
:10016000D3D2AFC2CEE52A6007207449152A21B543
:100170007800790020742EE580307E01F430E502AD
:1001800078FF53DACF207E0343DA20307E0343DA50
:1001900010C2D8C271E580307E01F430E50279FFEB
:1001A000C3E89970CB306103752A18207403752A4F
:1001B00018885CD27020740DE52B6004152B21C5C6
:1001C00043DA01C2D82070024138A85C206102C223
:1001D00070207431C3E894F0400374F0F8E8C4541C
:1001E0000F28F87984B703024105C313C31387218D
:1001F000200802C313200A06C3C898F8410528F84E
:10020000500374FFF8C3E895655003E565F888224C
:10021000E52D54066022206B1FE536C333C333F847
:10022000E564C313C313F9C3952240028922E8256C
:1002300022F52250037522FF852224A824C3E52439
:1002400095614002A8618825E5667002417CC3E89B
:10025000AA669A5003E8FAE4F9EAC333FBE568F4C6
:100260005B29400D2567F8E56760021567400B4183
:100270007C0AC3E5679A5002056778FF882620CF7D
:100280000AD0E0D0D043E610D2AD32C2CF053A78E2
:1002900001E52A6005307402152AC3E55C9401402B
:1002A00005755F0041B7756000756900E55F240161
:1002B000F55F5003755FFFD0E0D0D043E610D2ADBC
:1002C00032C2AF53E67F7592FA7593FFC2607591A3
:1002D00004D2AF32C2AF53E6EFC2ADC0D0C0E0C06F
:1002E000F0D2D3D2AFA8FBA9FCC2D8307102613BD7
:1002F00053DACF207E0343DA10307E0343DA20D274
:1003000071E580307E01F420E5026112882789289A
:10031000A16853DACF207E0343DA20307E0343DA2C
:1003200010C2D8C271307402A1547800E580307ECA
:1003300001F430E502A154885CA13C53DACF207E61
:100340000343DA20307E0343DA10C2712061028158
:100350001453DACF207E0343DA10307E0343DA20D1
:10036000C2D8D27188578958C3E89555F8E995568F
:10037000F97B007E087A00C3E8948CE9940050056C
:10038000755B008106882178A2E6A8216055C3E844
:1003900094C8E994005008E4D2E4FB7A0A61E1C30E
:1003A000E89468E994015008E4D2E3FB7A0F61E134
:1003B000C3E894D0E994025008E4D2E2FB7A1E61CB
:1003C000E1C3E894A0E994055008E4D2E1FB7A3C4B
:1003D00061E1C3E89498E994085008E4D2E0FB7A1C
:1003E000787E00C3E89559FCE9955AFD30E70AECA0
:1003F000F42401FCEDF43400FD755B00C3EC9AEDD0
:100400009E5003755B018859895A85575585585602
:100410007802A13CC3E89527F8E99528F9307C02D9
:10042000A120307B02A120307A02A119207502811F
:1004300037E9FDE8FC8156E9C313F9E813F8307990
:1004400002A119E9C313F9E813F8307802A119E9F8
:10045000C313FDE813FC20612CC3EC941CED940243
:100460004002816DED701EC3EC94C850180529E55B
:0E0470002970021529C3E529940A5002A154EF
:10047E00755C00D270A154E529600215297888E6D2
:10048E00F97400207F087896B90302789EE624FA64
:10049E00FEE43400FFC3EC9EFCED9FFD9208B90311
:1004AE0010A2085007207609D27681BF307602C29C
:1004BE0076A2085016B9030DECF42401FCEDF434C9
:1004CE0000FD0204D978007900A120B90315EC33A0
:1004DE00FCED33FDC3EC940AFCED9400FD50047C5E
:1004EE00007D00C3EC94FFED9400400678FF790088
:1004FE00A120EC8572F0A4C5F0A2F733F879004084
:10050E000302053C78FF790002053CE9C313F9E8C4
:10051E0013F8307C0EE9600278FFC3E81338F8E474
:10052E003400F9C3E894FFE99400400278FF885C38
:10053E00D270206102A154741FF4552F4BF52FC2B7
:10054E0074EB7002D274752A18307403752A0A304F
:10055E006102A16820740353DAFE207403752B0622
:10056E00D0F0D0E0D0D0D2AD43E610327901020502
:10057E00987903020598790A020598791E02059862
:10058E00796402059879C80205987817E4D5E0FDDC
:10059E00D8FAD9F6227A147B780205BF7A107B8CB2
:1005AE000205BF7A0D7BB40205BF7A0B7BC802052C
:1005BE00BFE573D5E001227902E4C294D5E0FDC215
:1005CE0095D5E0FDD295D5E0FDD294D5E0FDE9209C
:1005DE00E002C29330E002C297E573D5E0FDE92058
:1005EE00E002D29330E002D2977496D5E0FDD9C9DD
:1005FE00EAF8D5E0FDD8FBDBB8C29422C37C007DBF
:10060E000075F00005F0EA33FAEB33FB50F6EB130E
:10061E00FBEA13FAC3E9FFE8FEE89AF8E99BF95002
:10062E0004EFF9EEF8B3EC33FCED33FDD5F0DFED6E
:10063E00F9ECF822E889F08A20D2D4F8A9F07B00F0
:10064E0030F70B7BFFF42401F8E9F43400F9E88568
:10065E0020F0A4ADF0F8E98520F0A4AFF0FEED2E69
:10066E00F974003FFA7C04C3EA13FAE913F9E813AC
:10067E00F8DCF48BF030F70AE8F42401F8E9F434EE
:10068E0000F9E889F0C2D4F8A9F02222C3E541139B
:10069E00F9E54013F8C3E54498F8E54599F9500C8F
:1006AE00C3E89480E994FF40160206D1C3E8947F14
:1006BE00E9940050030206D1787F79000206D178C2
:1006CE008079FF8849894A22E5492546F8E54A3569
:1006DE0047F9854A20E4300701F43548FA30E70936
:1006EE00C3EA94F0401502070FC3EA940F500302B9
:1006FE00070F78FF79FF7A0F02070F780079007ADB
:10070E00F0C3E5249561500AC374019524500B0281
:10071E00072DE54A20E70E02072DE54A30E7068849
:10072E004689478A482278A5E6FAC3E54933F8E5B3
:10073E004A33F9D142E930E70BC3E89480E994FFDC
:10074E004013E167C3E8947FE994005002E16778B3
:10075E007F7900E167788079FFE820E715C3E5230C
:10076E0098F84009C3E89401400302078E7801020D
:10077E00078EE8F424012523F8400302078E78FF44
:10078E00884B2278A6E6FAA847A948D142E930E775
:10079E000CC3E89401E994FF40160207C2C3E89423
:1007AE00FFE9940050030207C278FF79000207C2E6
:1007BE00780179FFE920E715C3E54B98F84009C3A6
:1007CE00E8940140030207E978010207E9E8F424FE
:1007DE0001254BF840030207E978FF88242278FFB1
:1007EE0020692879A1E76023E541601F74FF8541E8
:1007FE00F0848539F0306A0375F005A4F8C5F06011
:10080E000278FFC3E895645002A864886322C3E5AA
:10081E00409440E5419401E563500314012D0460BA
:10082E0002F563220208352275E890227883E6FFEE
:10083E0030EDF9A8BDA9BE0570C3E570940840520D
:10084E00757000E9FA79A0E76044EA7007E5716017
:10085E001B02086EC3E895716010E5715006600CBE
:0F086E001402087A0460F902087AE571F571C383
:10087D00946D401B7561C0C394044013756180C3B2
:10088D009404400B756140C3940440037561007579
:10089D00BB0822E561F460020561E570B4070375DC
:1008AD00BB1022743279A787F0A4C5F0A2F733F8F4
:1008BD00C3E895614002A86188228824882588268E
:1008CD008864227540007541F022C2AF75C820A81A
:1008DD00CCA9CDAA3A30CF010A75C824D2AFAB3B13
:1008ED00AC3C883B893CC3E89BF8E99C206908F93E
:1008FD0030660221E62140AD3D8A3DF9EA9DFA6060
:10090D000478FF79FFAE3EAF3F8B3E8C3FA83BA9ED
:10091D003CC3E89EF8E99FF9C3E54113FBE540139D
:10092D00FAE82AF540E93BF54150067540FF75415F
:10093D00FF218DAA40AB41AC40AD417E047F02C387
:10094D00EB9404400D1E1FC3EB94084005206A0272
:10095D001E1FC3ED13FDEC13FCDEF7C3EA9CFAEB8F
:10096D009DFBEF6009C3E913F9E813F8DFF7EA28F7
:10097D00FAEB39FB8A408B4150067BFF8B408B4154
:10098D00C3EB94025002D2663069047F0321B8781C
:10099D0092E6FFC3E537948240110FC3E53794A06B
:1009AD0040010FC3EF940640027F057E02E541C46E
:1009BD00540FF9E541C454F0F8E540C4540F28F83C
:1009CD00C3E89EFAE99400FB4009C3EA9402EB9454
:1009DD000050047A02E4FB4132AA40AB41EBC4FE65
:1009ED00EAC4540F4EFCC3EA9CFAEB9400FBC3E837
:1009FD0013C313F8EA28FAEB3400FB8A408B41C38A
:100A0D00EB94024002C2667802EBC4FE7B00EAC49E
:100A1D00540F4EFAC3EA98FA4005C3940250027A75
:100A2D00027892E6FF3060024132855192855293F1
:100A3D00D26043E680C3E49AF8E49BF93066024144
:100A4D00BEE8FAE9FBD3E913FDE813FC885189529E
:100A5D00C3EF94036038EF20E00DE82CF8E93DF981
:100A6D00ECFAEDFB020A87E828F8E939F9C3E82426
:100A7D0002F8E93400F97AFE7BFFC3EF9403400ED0
:100A8D008A538B54884D894E8C4F8D5041F288532B
:100A9D0089548A4D8B4E8C4F8D503069127553F0A1
:100AAD007554FF754FF07550FF7551F07552FF413C
:100ABD00F2E8FAD3E813FC8851C3EF94036020EFFA
:100ACD0020E007E82CF8ECFA41DEE8282402F87A59
:100ADD00FEC3EF940340088A53884D8C4F41F28832
:100AED00538A4D8C4FE568C3335002646BF5683003
:100AFD00600241FC753402D26043E680E52D540658
:100B0D006034A840A941C3E913F9E813F8C3E91308
:100B1D00F9E813F8306904E92440F9C2AF53E67FD0
:100B2D00759100C3E498F594E499F595759104D207
:100B3D006043E680D2AF22D2647543007520003049
:100B4D006C03752040020B63D26475430075204021
:100B5D00306C0375200078017901206620E52D5455
:100B6D00066002C2647914E541C313700104F8C331
:100B7D00941440027814306904781B791B2060109E
:100B8D00E543600C306903D53404D26D810D7104D9
:100B9D000543E59B5440B5200261F730690908C350
:100BAD00E899400118618A20640A08C3E899400257
:100BBD006163618AC264C2AF53E67F75910030668E
:100BCD00127594007595F8759104D26043E680D244
:100BDD00AF6163E5417EFFC3334005C3334001FE82
:100BED00C3E49E759400F59561D4C3E5339401502B
:100BFD000261633064026163D802810B618AC26D48
:100C0D00C2AF53E67F7591008553948554957591C8
:100C1D0004854D92854E93D26043E680D2AFE52D8B
:100C2D0054066008206A020533020C49306D0D2010
:100C3D006C0A206407158115810215062278003093
:100C4D0064027801E53775F007A4F9E5F028F5F0B1
:100C5D00E9A2F013A2F113A2F213F537C394785061
:0F0C6D0003753778C3E53795384008D265D293C1
:100C7C00D295D2973060028180854F92855093D265
:100C8C006043E68022207D16C2AF754202C294D228
:100C9C0092306202C297D2AF759F10020E80C2AF23
:100CAC00754202C294D296306202C293D2AF759F43
:100CBC0010020E80307243207D20C2AF754203902B
:100CCC000132757B10D297C296306204C29581DED8
:100CDC00D294D2AF759F11020E80C2AF75420390B1
:100CEC000132757B10D293C292306204C29581FEA0
:100CFC00D294D2AF759F13020E80207D17C2AF75B0
:100D0C00420390010DD297306202C295D2AF759F0B
:100D1C0011020E80C2AF75420390010DD293306266
:100D2C0002C295D2AF759F13020E80207D16C2AF02
:100D3C00754204C292D296306202C295D2AF759FB0
:100D4C0013020E80C2AF754204C296D29230620278
:100D5C00C295D2AF759F11020E80307243207D2058
:100D6C00C2AF754205900121757B04D295C29430B7
:100D7C006204C293A184D292D2AF759F10020E80EE
:100D8C00C2AF754205900143757B40D295C2943039
:100D9C006204C297A1A4D296D2AF759F10020E80A6
:100DAC00207D17C2AF754205900103D295306202C7
:100DBC00C293D2AF759F10020E80C2AF75420590E0
:100DCC000117D2953062EBC297D2AF759F10020E0D
:100DDC0080207D16C2AF754206C296D29430620254
:100DEC00C293D2AF759F11020E80C2AF754206C27C
:100DFC0092D294306202C297D2AF759F13020E80CA
:100E0C00307243207D20C2AF754201900143757B47
:100E1C0040D293C292306204C297C12AD296D2AF0A
:100E2C00759F13020E80C2AF754201900121757B34
:100E3C0004D297C296306204C293C14AD292D2AF06
:100E4C00759F11020E80207D17C2AF754201900173
:100E5C0017D293306202C297D2AF759F13020E80E5
:100E6C00C2AF754201900103D297306202C293D295
:100E7C00AF759F11C26522900101757B00D293D290
:100E8C0095D297C292C294C296C26222788076FFA3
:100E9C000876FF0876FF0876FF08760308760408C4
:100EAC00760A087601087601087601788C760108B6
:100EBC0076FF0876FF0876FF0876FF0876FF08763F
:100ECC00030876FF0876FF0876FF0876250876D0AB
:100EDC000876FA0876FA0876040876FF0876010890
:100EEC00760008767A0876FF08760108760108768F
:100EFC0000087603087600227887E6FFC2727888AD
:100F0C00E6C394036008C27DE630E102D27DC27E66
:100F1C007889E630E102D27EC3EF94026008758EC8
:100F2C0001D273020F37758E00C273227880E614DB
:100F3C009000809378A5F67881E6149000809378E1
:100F4C00A6F67886E61490008D9378A7F67886E658
:100F5C00F539C394025003753902789CE67538FF55
:100F6C00B402037538A0B4030375388278A3E61471
:100F7C0090009A93F566D18322227896E6FA7897B8
:100F8C00E6FB7888E6B40305C3EB940EFB307F04D4
:100F9C007A007BFFC3EB9AFCC3948250027C82756F
:100FAC0072000572EC8572F0A4C3E5F0947D40F2FA
:100FBC0022D27FF1861205891205897A007B007C8A
:100FCC001012057FE55C2AFA74003BFBDCF37C0411
:100FDC00C3EB13FBEA13FADCF7FEC27FF186227532
:100FEC007C00757D00E5EF20E60375200005209060
:100FFC003FFFE520146006901DFF14600093046011
:10100C000375EF1653D9BF7581C043FF8012057A63
:10101C0075EF0643B203E5B3240220E70DF521E595
:10102C00E320E0068521B343E301120E837580FFB4
:10103C0075A40075F1B275D4DF7590A975A5FC7512
:10104C00F2FC75D50175A60175E241120E83E4F828
:10105C00F6D8FD756801120E98121557789886739C
:0E106C00753001C2AF1205931205A31205895B
:10107A001205AA1205891205B112058912167412EF
:10108A00059312059312058EC2AF757C00757D001B
:10109A0078FA79FA308507D9FBD8F7021C00120FC3
:1010AA0004120F38120F85120F8678988673120E63
:1010BA008375881075890275C82475910475D8409E
:1010CA0075A82275B80275E690759B80759D0075A6
:1010DA00D10E75BC5875BB0875BA1175E880120532
:1010EA007AD2AF12083275360053DACF207E034324
:1010FA00DA20307E0343DA1043DA01C2D8C2711211
:10110A000593D2617B037A0CE55B70077A0CDB03EB
:10111A00021092120589207003021092C270E55CD7
:10112A00C3940240E1E52F541F855E5DF55EB55D0F
:10113A00D5DAD5C26153DACF207E0343DA20307E76
:10114A000343DA10C2D8C27178A2E67008D274E5F5
:10115A002F54E0F52FC27575290012058E307409D7
:10116A00C3E529940A4002D27512057F78023074C9
:10117A00027800C3E55C9840F0C2AF1205A31205DD
:10118A00A31205A3D2AF120593754C007888E6B472
:10119A000302419212057F788CE6C3940150030240
:1011AA001292E530C394015003021292757CA57520
:1011BA007DF1207435C3E55C94FF5003021292C29C
:1011CA00AF1205B8D2AF12058EC3E55C940150EF99
:1011DA00C2AF1205A31205841205A3D2AF12058E5F
:1011EA00C3E55C94FF40E90216F97F05D27F120F2E
:1011FA008612058EC2AFC27F120F86AE5CC3E55C53
:10120A00947FD2AF500241A212057AC2AF1205B83A
:10121A00D2AFDFD8120FBDC3EE94057897F6120548
:10122A009312167C7F0AD27F120F8612058EC2AFE6
:10123A00C27F120F86AE5CC3E55C947FD2AF50E4E6
:10124A0012057AC2AF1205A31205841205A3D2AF02
:10125A00DFD4120FBDEE24037896F6F87997E7C328
:10126A0094824003985006E824827897F6120593F0
:10127A001215991216AB12058E120F86C3E55C94ED
:10128A00FF500221B60216F9757C00757D00C3E590
:10129A005C954C4003855C4C12058E78017988E791
:1012AA00B403027805C3E55C9840022196C2AF12E6
:1012BA0005B81205B81205B8D2AF120593753000F9
:1012CA00E4F531F5320531E531F4703F0532789AAB
:1012DA00E67819146012783214600D787D1460086B
:1012EA0078FA146003753200C3E53298401D120E75
:1012FA008312057A153275310078998673C2AF1256
:10130A0005B8D2AF7898867312058E120584E52A3D
:10131A007005307402019278012074027806C3E5E0
:10132A005C9840A17888E6C39403600312058EE5B1
:10133A002A7003021092C2AF120E83E4F522F5233B
:10134A00F524F525F526F567D2AF7885E6C333F59A
:10135A0065E4F544F545F546F547F548F570F52C8D
:10136A00F52DF53775700875BB1012057A12083617
:10137A0030EDFDA8BDA9BEE97001F8887112083ADE
:10138A0075700875BB10120F04C2AF7561FF1208A1
:10139A00B0852261852262852263D2AF75220175EA
:1013AA002401752501752601856069756A017888A9
:1013BA00E6B40307C27D307602D27DD268D269755F
:1013CA003300120DDD120E0C1208D01208D71208C3
:1013DA00D01208D71208D0120B55120699120C4ACD
:1013EA00120C911208D7120B44306E0312069A207F
:1013FA0066031207EC30660312081C120C4A120C20
:10140A00C01208D7120B55306E031206D6120C4AB8
:10141A00120D371208D7120B44306E03120734121A
:10142A000C4A120D661208D7120B55306E031207BA
:10143A0091120C4A120DDD1208D7120836120B440B
:10144A00120C4A120E0C12083A1208D730692F856C
:10145A006461856462856069756A0179187A0CC36A
:0E146A00E53399400CC269D26A8A357561FF7C
:10147800021488C3E55C940140030213E102150ECF
:10148800306A1D206C1AE535147006C26AD26B6189
:10149800E1F535C3E55C940140030213E102150E42
:1014A800753600788279A4E760027803C3E55F980F
:1014B8005054307404E52A604D7888E6B403172048
:1014C8007D0520760781DE30760281DE206C07D22A
:1014D8006C856461812078F0306C058564617820C2
:1014E800C3E54198500261E1306C1BC26CC27D308B
:1014F8007602D27DD26A75351285646161E105365E
:10150800E55C6002A111753600C2AF120E837887C0
:10151800E6FE7602120F047887EEF6E4F522F5234C
:10152800F524F525F526F565752C00752D00D2AF47
:1015380012058E120E8378A4E66006C293C295C285
:1015480097307409C3E53694044002019241CA9069
:101558001A0D78201215DBE520B45A0CA31215DBFE
:10156800E520B4A503021579120E981215990215F3
:1015780098901A0378807B0A1215DBA308DBF99090
:101588001A0F788C7B191215DBA308DBF9901A283F
:1015980022C2AF12161E1215FB901A00740E1215F5
:1015A800E0A374071215E0A374151215E0901A034E
:1015B80078807B0A1215DFA308DBF9901A0F788C64
:1015C8007B191215DFA308DBF912163112160F90DA
:1015D8001A2822E493F622E6438F01538FFDFFC3B6
:1015E800E583941C400122EF857CB7857DB7F053D5
:1015F8008FFE22438F02438F01857CB7857DB7908C
:101608001A0DF0538FFC22901A0D745AB1E0901AFB
:101618000E74A5B1E0227A3079D07820901A40B1C2
:10162800DBE520F709A3DAF7227A3079D0901A405F
:10163800E7B1E009A3DAF922AB74A875BB01027916
:1016480084BB02027985BB03027986BB04027992C6
:10165800BB05027987BB060279A3BB0702799CBB4D
:1016680008027988BB09027989E8F7227C05120506
:1016780093DCFB22C2AF1205A31205AA1205B11210
:1016880005B81205841205A31205AA1205B11205A0
:10169800B81205841205A31205AA1205B11205B8DD
:1016A800D2AF22C2AF1205B81205B11205AA1205AF
:1016B800A31205841205B81205B11205AA1205A3D2
:1016C8001205841205B81205B11205AA1205A3D293
:1016D800AF22AE74AF75C2AF1205A31205A31205EF
:1016E800A3120584DEF21205B8120584DFF8D2AF22
:1016F80022D17CD174D17475740175750175760029
:10170800D1DA7C05AD5C120593C3ED955C70F5C329
:10171800E55C9401400AC3E55C94FF40320217354A
:10172800D140B199D17CC2AF75EF16D174DCD50523
:1017380076C3E5769403500280C6D1740575E574C6
:101748001490009F93F808C3E57598500280AED1B5
:1017580074D1740574C3E574940A5002809C120E07
:0A17680098B199C2AF75EF16D17465
:0319FD00020FEBEB
:101A00000E0715FFFFFFFF03040A0101015AA5019C
:101A1000FFFFFFFFFF03FFFFFF25D0FAFA04FF01DE
:091A2000007AFF0101000300FF40
:101A400023476175694745313833313841232020B8
:101A500023424C48454C4923463333302320202031
:101A60002020202020202020202020202020202076
:101C0000C2AFC2D353D9BF7581C043B20343FF8073
:101C1000752438752503B1DC7529A5752AF175E29F
:101C20004043F12053A4DF75D4FFD2857DFA7803B9
:101C300079E67C10752200752300901DE97B0675FE
:101C400024987525013085028145208508D8FBD967
:101C5000F9DCF781B7308508D8FBD9F9DCF781B713
:101C6000B19CE493A3C39A6004DDC381B7DBDBB10D
:101C70008E6002812E7B08E493FAA3B16FDBF87AC1
:101C800030B16F752200752300B18EEAFCEBFDC305
:101C9000ED94FE400EB18E8A278B28ED30E0048A49
:101CA000828B83B18E7AC270D8C3ED94FE601950D6
:101CB000CEBD002BEC600F7520007521FF7529004B
:101CC000752A000200008100A827A9280809D80465
:101CD000D90281DCB192EA89AAF281CE0D81A3C337
:101CE000ED94035053EDA2E092007AC5C3E58294CF
:101CF00000E583941C508A200010438F02438F011B
:101D00008529B7852AB7F0300029A827A92808090E
:101D1000438F01538FFDD804D902A133C3E58394C7
:101D20001C4003A3A11689AAE28529B7852AB7F02A
:101D3000A3A116538FFC817F7AC1BD030CE493A34A
:101D4000FAB153DCF8B14B817F8181AA22AB23B178
:101D50006FEBFAEA6222752608C3E52313F523E543
:101D60002213F52250066323A0632201D526EAB18F
:101D7000DCB1DC75260AEAF4200102D285300102CA
:101D8000C285B1DCC3134002C201D526EB22B19259
:101D9000EAFB208502A192308502A197752608AE44
:101DA00024AF25C3EF13FFEE13FEB1E0B1DCC3EAAD
:101DB000133085024480FA30E703632201C3E52330
:101DC00013F523E52213F52250066323A0632201B5
:101DD000D526D9E52265236523F52222AE24AF2539
:101DE0000E0FDEFEDFFCD20122424C48656C6934E6
:071DF000373163F3300601F7
:00000001FF
